:0400000028C0FECF47
:10000400FDCFFCCF84C2FACF97C0F8CFF7CF70C032
:10001400F5CFF4CFF3CFF2CFF1CFF0CFEFCFEECFD8
:10002400EDCF88EB92C2E1C484EA80C0FFF78395E8
:10003400A0BF898F9C979DA7B4FFB78707000000D6
:100044000000000000320A00040040000000F894A0
:10005400EE27ECBBF1E0FBBFEBBFE5BFF8E1F1BD80
:10006400E1BD8DE0A2E0BB27ED938A95E9F780E03E
:1000740094E0A0E6ED930197E9F7EAE4F0E08591D6
:100084009591009761F0A591B59105901590BF01E8
:10009400F00105900D920197E1F7FB01F0CFEFE538
:1000A400EDBFE4E0EEBFC0E6D1E0E8C2AA931A9344
:1000B40010E01830D0F4FCD5E03039F4E981E09553
:1000C400E07811F4C39801C0C39AF2D5E13030F05E
:1000D400E981E07811F4C39801C0C39AC59AE98113
:1000E400EE0FE983C5981F5FE4CF18812296089527
:1000F400E3D5EC2DA1E020D8AE2FECD5EFD5A0812F
:10010400E9D5EF55FE4FA081D1DFC49AC498C394BA
:10011400E7E0EC1508F4CC24A3C2AA93E881E064D8
:10012400E7B98BE18A95F1F7369A349BFECF349A7E
:10013400E4B1F5B1219608951895D3D511F0D6D52B
:1001440009F008C0CED511F0D1D509F003C0E1E023
:10015400E0938601C6D511F4C9D509F453C0E0E093
:10016400E0938601E1E0E71539F4A2D5C3D5E23086
:1001740018F0A0E0B0E0C1D5E2E0E71519F0E7E03F
:10018400E71531F4BDD5C3D5E43010F0B9D5B5D5F4
:10019400E3E0E71519F0E8E0E71539F4BAD5B7D587
:1001A400E73118F0B6D5EAE036D8E4E0E71519F0FF
:1001B400E9E0E71531F4B4D5AAD5EA3010F0B0D5AA
:1001C400B6D5E5E0E71519F0EAE0E71531F4B2D564
:1001D4009ED5E23010F0AED590D5B3D511F0B4D59C
:1001E40031F4B5D594D5E23010F0B1D586D5B6D575
:1001F40011F4B7D509F003C0E0E0E0936001AEE587
:10020400B1E08CD7B1D511F0B4D509F008C0ACD5A4
:1002140011F0AFD509F003C0E1E0E0938701A4D564
:1002240011F4A7D509F42BC0E0E0E093870196D53B
:1002340011F497D509F005C0E0E0E0936101E09383
:1002440060018CD528F473947FD510F4E1E07E2E00
:1002540085D511F486D508F006C0E6E48E2E939475
:100264008CD508F49924A8E3B0E08AD511F48BD591
:1002740009F002C0E4E09E2EA6E2B2E04FD786D594
:1002840011F089D509F008C081D511F084D509F0A1
:1002940003C0E1E0E093880179D511F47CD509F439
:1002A40015C0E0E0E093880159D511F45AD509F05E
:1002B40003C0E0E0E093610151D510F452D509F098
:1002C40002C077249924AEE5B1E028D747D511F4CC
:1002D4004BD509F010C06394E4E6E61558F4E1E068
:1002E4009E2EA7E3B0E04CD511F459D509F002C015
:1002F400E2E09E2E0FC032D521F4F3D411F446D59A
:1003040009F007C06394E8ECE61510F4E1E07E2EF2
:1003140001C06624E6D411F424D508F073C042D594
:10032400E23010F443D508F41DC039D519F441D591
:1003340044D508F002C03DD544D53BD546D518F088
:10034400AEE1B0E046D549D519F44AD536D508F022
:1003540002C046D536D544D538D518F0AAE2B0E067
:1003640038D516C01CD531F424D5BF011BD53CD5D6
:100374003DD508F002C01DD524D52FD531F430D594
:10038400BF0110D531D532D508F002C029D519D511
:1003940038D5E23010F439D508F41DC0F4D419F47A
:1003A40037D50BD508F002C033D50BD531D50DD5D3
:1003B40018F0A0E2B0E00DD5E0D419F42DD5FDD4A9
:1003C40008F002C029D5FDD427D5FFD418F0ACE23B
:1003D400B0E0FFD414C0D7D429F41AD5BF0111D585
:1003E4001FD508F002C014D5ECD4C7D429F414D511
:1003F400BF0107D515D508F002C00ED5E2D4AD2D46
:10040400BB278CD6C3D411F4ACD408F023C0C7D412
:1004140019F4CFD411D508F002C0CBD410D5DDD453
:1004240019F4DED409D508F002C0DAD408D5ABD467
:1004340019F4EED401D508F002C0EAD400D59DD455
:1004440019F4EAD4F9D408F002C0E6D4F8D4AD2DF6
:10045400BB2764D6E1E09E1680F043D421F084D417
:1004640011F094D441F4E6E48E2EE4E6ED1510F494
:10047400EAE0DE1A02C0EEEEDE2EB394EAE7EB15F4
:1004840010F4EFE701C0EFEFAE2EEAE5EB1521F42F
:10049400E1E0E81508F48A94E1E0E81511F4882411
:1004A400992408957FD4E23038F480D428F0CBD452
:1004B400A83EE3E0BE0708F403C0E7EEF3E0C8D4C7
:1004C400A2E1B0E05DD411F071D410F4E1E001C018
:1004D400EAE0E093900195D4E23038F496D428F021
:1004E400BCD4A83EE3E0BE0708F405C0E0E7F1E0B1
:1004F400A7EEB3E0B7D4A3E1B0E042D411F085D4C1
:1005040010F4E1E001C0EAE0E09391010895D4D34E
:10051400E52D5394E41508F443C05524A6D4A091C2
:100524006201B09163011DD693D4A0916401B0918E
:1005340065019BD416D6E0937001F093710197D4B2
:1005440094D40FD6E0937201F093730195D48DD4B3
:1005540008D6E0937401F093750193D486D401D640
:10056400E0937601F093770191D47FD4FAD5E093A8
:100574007801F0937901E0E0E0936201E093630194
:10058400E4E6F1E088D4E6E6F1E085D4E8E6F1E0DB
:1005940082D4EAE6F1E07FD4ECE6F1E07CD460C0FA
:1005A400A8E1B0E0EDD370F401D420F077D47AD48C
:1005B4007DD402C073D476D4A0916201B09163015A
:1005C4007BD40DC0F3D320F07ED46CD46FD402C09E
:1005D4007AD468D4A0916201B09163016DD4A9E189
:1005E400B0E0CED370F411D420F075D45BD477D4BA
:1005F40002C071D457D4A0916401B091650175D43F
:100604000DC003D420F078D44DD469D402C074D47E
:1006140049D4A0916401B091650167D4A0E074D479
:1006240026D47BD4E0936601F0936701A5E075DDE1
:1006340077D422D472D4E0936801F0936901A3E0E3
:100644006CDD6ED41ED469D4E0936A01F0936B011F
:10065400A1E05AD41BD461D4E0936C01F0936D01F2
:10066400E991EFBFF991E991B991A9919991899192
:1006740079916991F990199009901895E0E0E5BB9A
:10068400E4BBE8BBEFE3E7BBE7E0E2BBE8EFE1BBD9
:10069400E3E0E3BFE0E0E2BFEFBDE3E0EEBDE0E0B6
:1006A400EDBDECBDE7BDE6BDEEE1EBBDE5E8EABDC1
:1006B400E0E0E9BDE8BDE2BDE6E0E5BDE0E0E4BDC3
:1006C400E3BDE5BFE1E5E9BFE0E0EAB9E0E8E8B9A8
:1006D400E0E0E0BFE0ECE7B9E3E8E6B9E0E0EDB97B
:1006E400E6BFE8EC7E2E789428DDDCDEE8ECE71546
:1006F40049F5E0E3F0E004900092A801E8E3F0E0BB
:1007040004900092A701E8E2F0E00DD4E093A60182
:100714000DD404900092A5010CD404900092A00181
:100724000BD401D4E0939F01E6E3F0E0049000923F
:100734009E01FFD3F8D3E0939D01ADEDB7E0EED475
:100744007724D2C0FED211F0FFD209F455C0D8D21A
:10075400F6D391F4F7D3F9D3FED308D411D420D42B
:1007640021D4F9D325D42ED430D436D438D42AD4B1
:100774003DD4F1D341D445D4C3D202D3E8F145D416
:10078400E436A0E0FA0718F4BBD248D408F405C054
:10079400D9D3DBD346D4E49105C0D4D3D6D3DBD3A9
:1007A40007D4EED3EC9331D43A9720F4A9D21FD5D1
:1007B400E33008F405C0C6D3F5D333D4E49110C0B4
:1007C400C1D3F0D3C8D308D40AD404902CD431961E
:1007D400DF0129D4A2D3E557FE4FE081E021DB01FC
:1007E400EC93B0D3F2D308D4EDD300D40F0191D25B
:1007F4001DD4E491D001EC93B1D211F4B2D209F03A
:1008040073C011D418D4EA5FFF4FDF0198D3E9F421
:1008140099D317D419D40FD419D4A8D31FD4C0D3BF
:1008240023D412D408D412D4C3D3CCD3E256FE4F6B
:100834000BD401D40BD4D0D3D2D3C4D3E356FE4FBC
:1008440003D4F9D303D4D8D3DCD3EDD3F4D3EA5F00
:10085400FF4FDF0195D208F447C0E5D3ECD307D4AA
:10086400E436A0E0FA0728F4D001AA5FBF4FD6D33C
:1008740008F405C067D3E5D3D4D3E49107C062D3A9
:10088400E0D3E2D3D8D3E2D393D3E8D3EC93CBD35E
:10089400D2D3EDD33A9730F4D001AA5FBF4FA7D497
:1008A400E33008F405C04ED3DFD3BBD3E4910CC0CE
:1008B40049D3DAD3C9D3BFD3C9D38ED390D3A491A8
:1008C400E0918E01EA23DB01EC933CD3D8D3BCD373
:1008D400B2D3BCD391D376D3D5D3B6D3ACD3E45F60
:1008E400FF4FDF01A3D38DD32CD210F076D210F4B6
:1008F400CCD301C0CFD3E0939601E1E0E71511F426
:10090400949A01C09498A6E0B0E088D320F4EFE76D
:10091400E0938B0109C0EFEFE0938B01A6E0B0E018
:100924007DD311F4EFE701C0EFEFE0938C01A7E072
:10093400B0E074D320F4EFE7E0938D0109C0EFEF4A
:10094400E0938D01A7E0B0E069D311F4EFE701C0B3
:10095400EFEFE0938E01992051F4E0916E01F09154
:100964006F019CD3E0917001F091710112C017D214
:1009740011F41FD293D331D211F432D28FD303D2D4
:1009840029F446D2E0937C01F0937D01F6D129F459
:1009940043D2E0937C01F0937D0101D211F0F3D1B5
:1009A40071F4D0D24ED33DD37ED35ED37ED367D3FE
:1009B40080D379D367D335D3E491EA21EC930DD274
:1009C40011F0DBD159F4BED23CD36FD34DD375D3E0
:1009D40056D373D357D325D374D3EC93E1E0E715FF
:1009E40011F5B0D22ED3DF01E1E3F0E05CD33CD3C8
:1009F400DF01E6E2F0E0E491EC935AD1E03031F427
:100A0400A1D23DD3DF01E8E3F0E004C09BD237D3A9
:100A1400DF018FD2E491EC9395D234D3DF01E1E38B
:100A2400F0E0E491EC93E2E0E71519F0E7E0E71574
:100A340099F488D206D348D336D316D347D341D3B7
:100A4400AFD21DD3BF015CD1D2D3CED1319642D324
:100A540019D3E7D268D2EC93E3E0E71519F0E8E0A4
:100A6400E715A9F46FD2EDD2DF01EBE2F0E01BD37E
:100A7400FBD236D326D394D202D30F014AD1D6D295
:100A8400E491D0018DD2FED2CCD24DD2EC93E4E0ED
:100A9400E71519F0E9E0E71589F454D2D2D20DD361
:100AA400E3D207D30ED37CD2EAD2BF0139D19FD38C
:100AB4009BD110D3E7D2B5D236D2EC93E5E0E7155B
:100AC40019F0EAE0E71591F43DD2BBD209D3EBD299
:100AD400CBD2EFD2F6D264D2D2D2BF012BD187D3FC
:100AE40083D1F8D2CFD29DD21ED2EC932AD110F06A
:100AF40074D110F4CAD201C0CDD2E093960121D1B1
:100B040011F022D1D9F58FD2E95CFF4FDF0117D262
:100B140081F418D21AD2DF010CD2C5D243D2D6D274
:100B2400C2D2E2D2D1D2BFD261D2DF01EFE3F0E090
:100B340010C008D20AD2C8D2B6D234D2DF01EEE352
:100B4400F0E0B1D2D1D2CCD2AED250D2DF01EFE2BA
:100B5400F0E0E491EC93F6D174D2DF01EFE3F0E03E
:100B6400A2D282D2B3D29FD28AD2AED29CD28AD21D
:100B7400DF0159D2E95DFF4FE491EC93A7E3B0E0C4
:100B8400DED1D1F416D10F012BD1E015F10550F0CF
:100B940010D159D1AFD208F0C19A22D1AED208F007
:100BA400C19809C006D1A9D208F0C19A19D14BD174
:100BB400A1D208F0C1980DC013D19FD218F0E1E082
:100BC400E0936001A0916001A13011F4C19801C0CB
:100BD400C19AA8E3B0E0B3D1F1F41AD10F011CD14A
:100BE400E015F10560F014D138D184D208F0C29A2E
:100BF40013D133D1AE17BF0708F0C2980BC008D188
:100C04002CD1AE17BF0708F0C29A06D126D172D2F2
:100C140008F0C2980FC000D120D1AE17BF0718F05A
:100C2400E1E0E0936101A0916101A13011F4C29867
:100C340001C0C29AA6E3B0E0DAD2E530A8F1219768
:100C4400E0E0E883E883A881A63008F55AD2A050F2
:100C5400B0406DD056D2AA5FBF4F69D052D2A45FC4
:100C6400BF4FE1E1D8D24DD2AE5EBF4F60D049D282
:100C7400A85EBF4F42D0E881AEE1B0E045D2E88142
:100C8400AAE2B0E041D2E881EF5FE883DCCFA6E3DB
:100C9400B0E0E3E0C0D2A7E3B0E02FD0A8E3B0E037
:100CA4002CD0ACE339D22196A1E036D21DCDFFCFB2
:100CB400A0E0B0E09CD208950A921A92FA926A9344
:100CC4007A938A939A93AA93BA93EA93FA93EFB78F
:100CD400EA930895EBD9EC2DF0E00895E356FE4F26
:100CE4000895A0E08299A1E0A0300895A091860122
:100CF400A0300895EF5F8FD20895E0E08CD208957C
:100D0400E0919601F0E0EA5FFF4FDF0108956FD2B2
:100D1400F1CFE0919601F0E0E45FFF4FDF01089529
:100D2400E0919601F0E0EE5EFF4FDF010895E1E00F
:100D340072D20895E0919601F0E0E85EFF4FDF0182
:100D44000895E6E0E7150895EBE0E7150895E091CE
:100D54009601F0E0E95CFF4FDF010895E0E0E7155C
:100D64000895E0E0E9150895A0E08199A1E0A0309C
:100D74000895A0918701A0300895E4E0E91508954D
:100D840036D2E1300895E3E0E9150895A0E08099B2
:100D9400A1E0A0300895A0918801A0300895E1E079
:100DA400E9150895A2E1B0E022D20895A6E0B0E0EA
:100DB400E7CFAEE1B0E017D20895E73EA3E0FA072B
:100DC4000895319620D231970895E83EA3E0FA07BA
:100DD4000895E4E8F3E017D20895E2E0E9150895F0
:100DE400AAE2B0E000D20895F0E00895AFEFB3E0D6
:100DF400B3D1DF01E0919001F7DFC6D16E177F0711
:100E04000895A3E1B0E0F3D10895A7E0B0E0B8CF2E
:100E1400A0E2B0E0E8D10895ACE2B0E0E4D10895F6
:100E2400E3DFAFEFB3E098D1DF01E0919101DCDFC4
:100E3400ABD16E177F070895DF01FED10895319776
:100E4400E2D131960895A0916E01B0916F01089599
:100E5400E0936E01F0936F010895A0917001B09139
:100E640071010895A083B1830895E42DBDCFA091AD
:100E74006601B09167010895A0916801B09169017C
:100E84000895A0916A01B0916B010895A0916C013D
:100E9400B0916D010895A0E0B0E0E4CFA0E03DD9A9
:100EA4000F0180CFA1DFD0014FD10895DF01E09180
:100EB40090019ADF56D10895EA0FFB1FE093620177
:100EC400F09363010895A0E028D9AFEFB3E0AE1B1F
:100ED400BF0B0D0167CFA1E020D90F0192CFDF0135
:100EE400E091910181DF3DD10895EA0FFB1FE0936A
:100EF4006401F09365010895A1E00FD9AFEFB3E069
:100F0400AE1BBF0B0D017DCF08D9AFEFB3E0AE1B15
:100F1400BF0BE2E0F0E018D10895EA0FFB1F08953B
:100F2400EE0FFF1F0895E491EF770895E0E3F0E0FA
:100F34000895E4E3F0E00895E3E3F0E0089557D181
:100F4400E0300895E09195014FCFABE0B0E044D19B
:100F5400EA1BFB0BC3CEBF01A0919601BB27AA0FCE
:100F6400BB1FA658BE4F34D1DF010895E8EEF3E06D
:100F7400F8D0DF01EAE0F0E00CD1EA5DFF4F08951C
:100F84000490E091960130DF3096DF01E091960104
:100F94002BDFC3DFE557FE4FE081E021DB0108953D
:100FA400EC93D0CFAAE0B0E017D1EA1BFB0B96CEAE
:100FB400E4E6F0E0D6D0DF01EAE0F0E0EAD0EA5D72
:100FC400FF4F0895E491DB01EBCFA9E0B0E004D139
:100FD400EA1BFB0B83DEBFCFEAE0F0E00895C1D04B
:100FE400DF01FADFD6D0EA5DFF4F0895A8E0B0E054
:100FF400F3D0EA1BFB0B72CEEFDFCBD0EA5DFF4FE1
:101004000895E491DB01EC930895A0919601BB2728
:10101400AA0FBB1FA658BE4FDBD00895E8D0E2301C
:101024000895DF0183CFE0919601DECEE0D0DCDECF
:10103400EA5DFF4F0895A1E0B0E0CED0EA1BFB0BC0
:101044000895E056FE4F0895BF01EDCFAAE7B1E041
:1010540067DFAE0FBF1FBCD0DF010895A491E091FC
:101064008D01EA23DB010895E156FE4F08950F0137
:10107400AAE7B1E055DFAE0FBF1FAAD00895E2562C
:10108400FE4F0895E356FE4F0895E8E0E09395017E
:10109400E1E00895E0E0E09395010895E0937A019A
:1010A400F0937B010895E4917BCFDF01E6E2F0E069
:1010B400FACFDF01EBE3F0E00895DF01ECE3F0E0C9
:1010C400F2CFE491EA210895DF0136CFDF01E7E3AF
:1010D400F0E00895DF0180DF5FD0EA5DFF4F72CF5B
:1010E400DF01E5E3F0E00895A9E0B0E075D0EA1B84
:1010F400FB0BF4CDEA17FB070895A5DEAE17BF0777
:101104000895A881B0E008956FDE0ADFAE0FBF1F17
:10111400E0E0F0E078D00895B0E000C0109639F037
:1011240080ED97E00197F1F7A8951197C9F7089515
:10113400F195E195F0400895EE230E2EEA2F19F073
:10114400EE0F0A94E9F70895FA9FF02DEB9FF00D46
:10115400EA9FE02DF10D08952DD0F6DF0EF4E8DFBF
:1011640008950024112490E1AA0FBB1F001C111C38
:101174000E1A1F0A18F40E0E1F1E01C0A1609A95C4
:1011840099F7FD01D001089515D0EBDF0EF4D0DFFF
:101194000895E7DFFD010895E894B7FF04C0A09522
:1011A400B09511966894F7FDC3DFDBDFFD010EF403
:1011B400BFDF0895E894F7FF02C0BADF6894B7FF71
:1011C40006C0A095B095119600F8039400FA08950E
:1011D400ED91FC91119708951B2EBF2FF12D1A2E1E
:1011E400AE2FE12D0895119602D0FE2F1197E199AB
:1011F400FECFFF93FFB7F894AEBBBFBBE09AEDB34D
:10120400FFBFFF91089507D01196EF93EF2F03D0FE
:10121400EF9111970895E19B02C0A895FCCF9FB769
:10122400F894AEBBBFBBE09A8DB3E81719F0EDBBE1
:10123400E29AE19A9FBF089500240A160B060895C6
:00000001FF
